:060000000C944D000C946D
:1000060000000C9400000C9400000C9400000C946A
:1000160000000C9400000C9400000C9400000C945A
:1000260000000C9400000C9400000C9400000C944A
:1000360000000C9400000C9400000C9400000C943A
:1000460000000C9400000C9400000C940000102793
:10005600E80364000A00010000100001100001001E
:1000660080C00000737065656420696E6465783AC7
:10007600202569004A616661726920262620426150
:1000860062616569000002006001660002006401A9
:1000960068000000F894EE27ECBBF1E0FBBFEBBF75
:1000A600E5BFF8E1F1BDE1BD8DE0A2E0BB27ED9330
:1000B6008A95E9F780E094E0A0E6ED930197E9F7E9
:1000C600ECE8F0E085919591009761F0A591B591E6
:1000D60005901590BF01F00105900D920197E1F78B
:1000E600FB01F0CFEFE5EDBFE4E0EEBFC0E6D1E007
:1000F6000C947D00609701E010E0E8E0EBBBEABB02
:10010600E0E0E8BBE7BBE5BBE4BBE2BBE0E2E1BBAA
:10011600E0E0E3BFE2BFECBFE1E8EFBDE1E0EEBD4A
:10012600E0E0EDBDECBDE7BDE6BDEBBDE0EAEABD56
:10013600E0E0E9BDE8BDE2BDE5BDE4BDE3BDE5BF88
:10014600E4BFE9BFE0E8E8B9E0E0E0BFE0E1EA9358
:100156000E944B03E6E9F0E00E949703829B0BC0E6
:10016600E4E6F0E00E949703829B03C0EAB5E550FF
:10017600EABD01E010E0839B03C0EAB5EF3F09F456
:100186000BC0E4E6F0E00E949703839B03C0EAB548
:10019600EB5FEABD01E010E0EAB5E33710F4E3E710
:1001A600EABDE1E0F0E0E017F10731F50E94E9026F
:1001B600FE01FA93EA93EAE6F0E0FA93EA93EAB5E7
:1001C600FF27662777270E94F00384E00E946402D7
:1001D6002896FE01FA93EA930E941903E0E0EA9357
:1001E600E1E0EA930E94D902EAE7F0E0FA93EA93A3
:1001F6000E94280300E010E0ADCFFFCF5F9BFECF4B
:10020600ECB108955D9BFECFE881ECB92196089587
:100216001A930A93AC81BD810E94E8033097D9F006
:10022600AA81BB810E94E8038F01309749F0023012
:10023600E0E01E0778F0F80131978F01ED93FC930B
:10024600AC81BD81ED91FD913196FE93EE93319790
:10025600AE81A08304C0EE81EA930E940501198154
:1002660008812796089526970E94F50310E0EA89EB
:10027600FB893196EA8BFB8B3197E4912E2FE03088
:1002860011F40C946002E12FE03039F4253211F4B8
:1002960011E002C00E949B030FC1E130A9F4253290
:1002A60019F40E949B0307C112E040E000E02D32E2
:1002B60011F401E001C12B3211F44BE2FDC02032F2
:1002C60011F440E2F9C002C0E23039F450E013E024
:1002D600203311F40068F0C004C0E33011F00C9430
:1002E6005F02203310F02A3308F009C0A52FEAE098
:1002F600EA9FF0015E2FE22FE0535E0FDDC0E22F92
:10030600E33631F40E94A603EC910E94AD03D3C0FC
:10031600E33741F40E94A6030E94B8030E948203B9
:100326001E2F0AC0E03761F40E94A6030E94B8039C
:100336000E948C031E2F086002600F7730E038C0E1
:10034600E43611F0E93611F4046002C0E53731F401
:10035600E4E5F0E0EE83FF8315E00DC0E83511F427
:10036600086004C0E83711F00C945E02EEE5F0E098
:10037600EE83FF8314E002FF15C00E94A6030E94CD
:10038600E803EA87FB87AA85BB8510972CF40E94B1
:10039600E403EA87FB874DE2403011F01F5F01C09E
:1003A6000B7F06C00E94A6030E94E803EA87FB872C
:1003B60000FD11C0151778F407FF08C002FF04C03E
:1003C6000B7F242F115001C020E301C020E20E94C0
:1003D6009B035150EFCF312F01FF1AC03030B9F0D7
:1003E60003FF08C0EE81FF813196EE83FF833197CC
:1003F600E49105C0AE81BF81ED91AE83BF83EA93E0
:100406000E94BF03503009F051503150E7CF4AC027
:1004160020E3EE81FF813296EE83FF8332970E94BE
:10042600EC03E887F987E885F985AA85BB85AE17C9
:10043600BF0750F02F5FA885B985EA85FB85EA1BC3
:10044600FB0BEA87FB87EFCF2A3328F003FF02C0B6
:10045600295F01C0295D04FD1AC0213320F4A88557
:10046600B985119709F409C0531710F000FF01C0B0
:1004760013C020E207FF0BC020E3006102FF07C0A4
:100486000B7F4A930E94BF03503009F051500E94DF
:100496009B03503009F051503150A885B985129709
:1004A60008F0B6CF00FF07C0503029F05150E0E207
:1004B6000E94AD03F9CF10E0DACE0E94FC036496E9
:1004C6000895FF92F82E22971A930A93DE010E944E
:1004D600E0038D01DE0116960E94E0030E94E80308
:1004E600EA83FB83DE0114960E94E0030E94E80380
:1004F600FA93EA931A930A93FE013696FA93EA93CD
:10050600E0E0F0E0FA93EA930E943601AA81BB810B
:10051600E0E0EC93198108812496FF900895FFE0AE
:10052600FA95F1F70895AAB3AF70AABBD99AD898ED
:100536000E949202DA9A0E949202A9B3DA980E9465
:100546009202DA9A0E949202DA98A7FDF1CF0895F4
:10055600A07FAB2BABBBDA9A0E949202DA980E947C
:1005660092020895D998AAB3A76FAABBBBB3BF706E
:10057600A8810E94AB02A881A2950E94AB02D99ADB
:1005860021960895DA9A0E949202E9B3DA980E94B7
:100596009202E07F08950E9492020E94C502AE2F49
:1005A6000E94C502D998E295EA2B08950E94960208
:1005B600E881F0E0E05AFE4FE081A981EA0FEA9374
:1005C6000E94B50259804880229608950E9496029C
:1005D600E2E0EA930E94B5020E949602ECE0EA93FA
:1005E6000E94B5020E949602E1E0EA930E94B502DB
:1005F600E0E04E2E5E2E0895EF93FF93A881689457
:10060600AA3021F0E8945394751438F44394E0E04A
:10061600EA934A920E94D9022EF085DFD89AA881E1
:10062600AA93A0DFFF91EF91219608951A93A981CD
:10063600BA81ED91A983BA831E2FE03021F01A9377
:100646000E94FF02F4CF188110C01A93E981FA8143
:100656003196E983FA833197E4911E2FE03021F039
:100666001A930E94FF02F2CF188123960895AA27B3
:10067600BB271197F1F70895D998AAB3A76FAABB1C
:10068600BBB3BF70A8810E94AB02D99A2196089588
:10069600DA98D8987880E881E058E0936201E8819A
:1006A600E054E09363010E94C9030E94C9030E94BB
:1006B600C9030E943A03E0E2EA930E943F030E94C4
:1006C6003A03E8E20E94CF03E4E00E94CF03E5E8A4
:1006D6000E94CF03AAB3AF70AABBD99A0E94CE02DA
:1006E600E53011F0E0E009C00E949602E6E0EA93E8
:1006F6000E94B5020E94E902E1E021960895A991BF
:10070600B991EE27FF276D91662311F03196FBCF45
:100716000895AA27BB27E991F9910590002011F0C9
:100726001196FBCFFD010895FA93EA930C94D40336
:100736002A93EF85F889FA93EA93FE013F96FA9396
:10074600EA930C940B01A889B9891497A88BB98BE5
:1007560014960895EA93EF85F889FA93EA93FE01D1
:100766003F96FA93EA930C940B010E94E803EE83FA
:10077600FF83FA93EA930895EF85F889FA93EA934B
:10078600FE013F96FA93EA930C940B010E943A03FA
:10079600E0E3EA930C943F03EA930E94B5020C94BB
:1007A6003A03E991F991309639F080ED97E0019797
:1007B600F1F7A8953197C9F708950024AF0DB01D3C
:1007C6000895F195E195F0400895ED91FC9111970A
:1007D60008950590F491E02D08957A936A93FA931B
:1007E600EA9308955A934A933A932A931A930A934B
:1007F60008955D814C813B812A8119810881089584
:00000001FF
